:10000000A305C304000A0F020F0EE2014F0B590BA8
:10001000650B710B7B0B850B990BA50BEF0BAB0BDA
:10002000B30BB80BBD0BC20BEB0BEF0B3F0C190A5C
:10003000400C4B0900084505000845040008A304CE
:10004000C3046C00240A2C006D00050C3E00040063
:10005000ED02270AFE02270A050C3E00EC02270AE1
:10006000000804000506310A3F0C2D00ED02360A97
:10007000080C2E002F0305063F0AEF04400AEF0587
:10008000410A0000270C2D00ED02440AEE023A0A54
:100090000507480A0008A304C3042F002504280C00
:1000A0002D00ED02510A080C2E0003042F03030655
:1000B0005A0A5D0A00002505600A250404000400B0
:1000C000270C2D00ED02620AEE02550A670A680A43
:1000D000690A000025052B0C2D00ED026D0A0008B1
:1000E000330C2600EE0C1601290006000A0C230929
:1000F000AA0C1601290006007D0A220C160129000F
:100100000600820A0C0C2B00770C2600870A880A4E
:10011000330C26008B0A8C0AEB02840AAA0C160107
:1001200029000600930A940A880C1601290006008B
:100130007D0C23097700C80C38001506A20A350685
:10014000B00AEF0B61006607A30A6606A50A010262
:1001500097000102030617023700F802A20ABD0A3F
:100160006100E607B10AE606B30A01029700010240
:10017000030617023700F802B00A17024B091702EC
:1001800039003903390339031F0C7901060CB90012
:100190001902B7000008EE0C290006000A0C23091A
:1001A000FF0C2900060000081D091506DA0A3506AD
:1001B000120BEF0B660461006607DC0A6606DE0AB6
:1001C000170281000307DB0A050C2100100C2B002D
:1001D000190281000307E80A610069040902740337
:1001E000730303070600190281000307F30A610085
:1001F000140466061405190281000307FB0A610056
:1002000069050902060065056606040B61006504C0
:10021000EB02E80AFC02E60A1D023C00FA02E60ACA
:100220001B090008E6046100E607140BE606160B3E
:10023000170281000307130B050C2100100C2B0083
:10024000190281000307200B6100E904090274030D
:100250007303030706001902810003072B0B6100DB
:100260001404E6061405190281000307330B61002C
:10027000E905090206006505E6063C0B6100650418
:10028000EB02200BFC021E0B1D023C00FA021E0BAF
:100290001B090008010C3A003C003109030A1B024B
:1002A0003A001D023C000F0C3300FF0C3400D4094F
:1002B000F10B1F0C3300FF0C3400D40913022F0084
:1002C0004B0914022F004B09F10B2F0C3300FF0CCC
:1002D0003400D40913022F004B0914022F004B09DC
:1002E000F10B1B023A001D023C003F0C3300FF0CD7
:1002F0003400D409F10B31090F020F0E400D330009
:1003000031090F023400D409F10B03041B032E0042
:1003100003042E0303042E030E021F061B023A00E1
:100320007F001D023C005F0C3300FF0C3400D40939
:10033000F10B6F0C3300FF0C3400D40913022F00B3
:100340004B0914022F004B09F10B7F0C3300FF0CFB
:100350003400D409F10B15024306EF0B1B09700999
:10036000010C3F00F10BCB091F091D097F00F10BA8
:10037000010C3500F00C3600F10B020C35000F0CAF
:100380003600F10B35024306CB0B300CD5014B097F
:10039000380C4B09D00B580C4B09580C4B09D00B9F
:1003A000200C4B09530C4B09580C4B092D0C4B09D5
:1003B000500C4B09470C4B094D0C4B09200C4B09B9
:1003C000560C4B09320C4B092E0C4B09300C4B09C7
:1003D000310C4B094A0B31090F023B00F10B160996
:0603E0004A0B18094A0B4C
:1004000004006100DF0C0200000C2400020C250037
:1004100026002700010C28000500FF0C290006001B
:10042000000C2A00070075007F00C80C3B00020C7E
:100430003D00540CA304C3044B09040C2B00A3047B
:10044000C3041B09A304C3041F09A304C3041D0997
:10045000A304C3041F09A305C304EB021F0AA304DA
:04046000C3044A0B7C
:021FFE00FD0FD5
:00000001FF
